 Brackets

 Timestamp is 56b152d7 (Wed Feb 03 04:07:35 2016)

 Preferred load address is 10000000

 Start         Length     Name                   Class
 0001:00000000 000000f8H .idata$5                CODE
 0001:000000f8 00000004H .CRT$XCA                CODE
 0001:000000fc 00000004H .CRT$XCZ                CODE
 0001:00000100 00000004H .CRT$XIA                CODE
 0001:00000104 0000000cH .CRT$XIC                CODE
 0001:00000110 00000004H .CRT$XIZ                CODE
 0001:00000114 00000004H .CRT$XPA                CODE
 0001:00000118 00000004H .CRT$XPZ                CODE
 0001:0000011c 00000004H .CRT$XTA                CODE
 0001:00000120 00000004H .CRT$XTZ                CODE
 0001:00000128 00002210H .rdata                  CODE
 0001:00002338 000000dcH .rdata$r                CODE
 0001:00002420 0000000cH .rdata$sxdata           CODE
 0001:0000242c 00000004H .rtc$IAA                CODE
 0001:00002430 00000004H .rtc$IZZ                CODE
 0001:00002434 00000004H .rtc$TAA                CODE
 0001:00002438 00000004H .rtc$TZZ                CODE
 0001:00002440 00006f08H .text                   CODE
 0001:00009348 00000014H .text$yd                CODE
 0001:00009360 00000224H .xdata$x                CODE
 0001:00009584 00000028H .idata$2                CODE
 0001:000095ac 00000014H .idata$3                CODE
 0001:000095c0 000000f8H .idata$4                CODE
 0001:000096b8 0000045aH .idata$6                CODE
 0001:00009b20 000000a6H .edata                  CODE
 0002:00000000 00000bb0H .data                   DATA
 0002:00000bc0 00000f40H .bss                    DATA
 0003:00000000 00000058H .rsrc$01                DATA
 0003:00000060 00000380H .rsrc$02                DATA

  Address         Publics by Value              Rva+Base       Lib:Object

 0000:00000000       __except_list              00000000     <absolute>
 0000:00000003       ___safe_se_handler_count   00000003     <absolute>
 0000:00000000       ___ImageBase               10000000     <linker-defined>
 0001:00000000       __imp__lstrcpynW@12        10001000     kernel32:KERNEL32.dll
 0001:00000004       __imp__lstrlenW@4          10001004     kernel32:KERNEL32.dll
 0001:00000008       __imp__lstrcmpiW@8         10001008     kernel32:KERNEL32.dll
 0001:0000000c       __imp__GetCurrentThreadId@0 1000100c     kernel32:KERNEL32.dll
 0001:00000010       __imp__DecodePointer@4     10001010     kernel32:KERNEL32.dll
 0001:00000014       __imp__GetCommandLineA@0   10001014     kernel32:KERNEL32.dll
 0001:00000018       __imp__GetLastError@0      10001018     kernel32:KERNEL32.dll
 0001:0000001c       __imp__HeapFree@12         1000101c     kernel32:KERNEL32.dll
 0001:00000020       __imp__IsProcessorFeaturePresent@4 10001020     kernel32:KERNEL32.dll
 0001:00000024       __imp__EncodePointer@4     10001024     kernel32:KERNEL32.dll
 0001:00000028       __imp__HeapAlloc@12        10001028     kernel32:KERNEL32.dll
 0001:0000002c       __imp__RaiseException@16   1000102c     kernel32:KERNEL32.dll
 0001:00000030       __imp__TlsAlloc@0          10001030     kernel32:KERNEL32.dll
 0001:00000034       __imp__TlsGetValue@4       10001034     kernel32:KERNEL32.dll
 0001:00000038       __imp__TlsSetValue@8       10001038     kernel32:KERNEL32.dll
 0001:0000003c       __imp__TlsFree@4           1000103c     kernel32:KERNEL32.dll
 0001:00000040       __imp__InterlockedIncrement@4 10001040     kernel32:KERNEL32.dll
 0001:00000044       __imp__GetModuleHandleW@4  10001044     kernel32:KERNEL32.dll
 0001:00000048       __imp__SetLastError@4      10001048     kernel32:KERNEL32.dll
 0001:0000004c       __imp__InterlockedDecrement@4 1000104c     kernel32:KERNEL32.dll
 0001:00000050       __imp__GetProcAddress@8    10001050     kernel32:KERNEL32.dll
 0001:00000054       __imp__Sleep@4             10001054     kernel32:KERNEL32.dll
 0001:00000058       __imp__ExitProcess@4       10001058     kernel32:KERNEL32.dll
 0001:0000005c       __imp__SetHandleCount@4    1000105c     kernel32:KERNEL32.dll
 0001:00000060       __imp__GetStdHandle@4      10001060     kernel32:KERNEL32.dll
 0001:00000064       __imp__InitializeCriticalSectionAndSpinCount@8 10001064     kernel32:KERNEL32.dll
 0001:00000068       __imp__GetFileType@4       10001068     kernel32:KERNEL32.dll
 0001:0000006c       __imp__GetStartupInfoW@4   1000106c     kernel32:KERNEL32.dll
 0001:00000070       __imp__DeleteCriticalSection@4 10001070     kernel32:KERNEL32.dll
 0001:00000074       __imp__GetModuleFileNameA@12 10001074     kernel32:KERNEL32.dll
 0001:00000078       __imp__FreeEnvironmentStringsW@4 10001078     kernel32:KERNEL32.dll
 0001:0000007c       __imp__WideCharToMultiByte@32 1000107c     kernel32:KERNEL32.dll
 0001:00000080       __imp__GetEnvironmentStringsW@0 10001080     kernel32:KERNEL32.dll
 0001:00000084       __imp__HeapCreate@12       10001084     kernel32:KERNEL32.dll
 0001:00000088       __imp__HeapDestroy@4       10001088     kernel32:KERNEL32.dll
 0001:0000008c       __imp__QueryPerformanceCounter@4 1000108c     kernel32:KERNEL32.dll
 0001:00000090       __imp__GetTickCount@0      10001090     kernel32:KERNEL32.dll
 0001:00000094       __imp__GetCurrentProcessId@0 10001094     kernel32:KERNEL32.dll
 0001:00000098       __imp__GetSystemTimeAsFileTime@4 10001098     kernel32:KERNEL32.dll
 0001:0000009c       __imp__HeapSize@12         1000109c     kernel32:KERNEL32.dll
 0001:000000a0       __imp__WriteFile@20        100010a0     kernel32:KERNEL32.dll
 0001:000000a4       __imp__GetModuleFileNameW@12 100010a4     kernel32:KERNEL32.dll
 0001:000000a8       __imp__LeaveCriticalSection@4 100010a8     kernel32:KERNEL32.dll
 0001:000000ac       __imp__EnterCriticalSection@4 100010ac     kernel32:KERNEL32.dll
 0001:000000b0       __imp__GetCPInfo@8         100010b0     kernel32:KERNEL32.dll
 0001:000000b4       __imp__GetACP@0            100010b4     kernel32:KERNEL32.dll
 0001:000000b8       __imp__GetOEMCP@0          100010b8     kernel32:KERNEL32.dll
 0001:000000bc       __imp__IsValidCodePage@4   100010bc     kernel32:KERNEL32.dll
 0001:000000c0       __imp__HeapReAlloc@16      100010c0     kernel32:KERNEL32.dll
 0001:000000c4       __imp__LoadLibraryW@4      100010c4     kernel32:KERNEL32.dll
 0001:000000c8       __imp__UnhandledExceptionFilter@4 100010c8     kernel32:KERNEL32.dll
 0001:000000cc       __imp__SetUnhandledExceptionFilter@4 100010cc     kernel32:KERNEL32.dll
 0001:000000d0       __imp__IsDebuggerPresent@0 100010d0     kernel32:KERNEL32.dll
 0001:000000d4       __imp__TerminateProcess@8  100010d4     kernel32:KERNEL32.dll
 0001:000000d8       __imp__GetCurrentProcess@0 100010d8     kernel32:KERNEL32.dll
 0001:000000dc       __imp__RtlUnwind@16        100010dc     kernel32:KERNEL32.dll
 0001:000000e0       __imp__LCMapStringW@24     100010e0     kernel32:KERNEL32.dll
 0001:000000e4       __imp__MultiByteToWideChar@24 100010e4     kernel32:KERNEL32.dll
 0001:000000e8       __imp__GetStringTypeW@16   100010e8     kernel32:KERNEL32.dll
 0001:000000ec       \177KERNEL32_NULL_THUNK_DATA 100010ec     kernel32:KERNEL32.dll
 0001:000000f0       __imp__MessageBeep@4       100010f0     user32:USER32.dll
 0001:000000f4       \177USER32_NULL_THUNK_DATA 100010f4     user32:USER32.dll
 0001:000000f8       ___xc_a                    100010f8     LIBCMT:crt0init.obj
 0001:000000fc       ___xc_z                    100010fc     LIBCMT:crt0init.obj
 0001:00000100       ___xi_a                    10001100     LIBCMT:crt0init.obj
 0001:00000110       ___xi_z                    10001110     LIBCMT:crt0init.obj
 0001:00000114       ___xp_a                    10001114     LIBCMT:crt0init.obj
 0001:00000118       ___xp_z                    10001118     LIBCMT:crt0init.obj
 0001:0000011c       ___xt_a                    1000111c     LIBCMT:crt0init.obj
 0001:00000120       ___xt_z                    10001120     LIBCMT:crt0init.obj
 0001:00000128       _MainGuid                  10001128     Brackets.obj
 0001:00000138       _MenuGuid                  10001138     Brackets.obj
 0001:00000148       _DialogGuid                10001148     Brackets.obj
 0001:00000158       ??_C@_1DE@BGKMIKPD@?$AAE?$AAu?$AAg?$AAe?$AAn?$AAe?$AA?5?$AAR?$AAo?$AAs?$AAh?$AAa?$AAl?$AA?5?$AA?$CG?$AA?5?$AAF?$AAa?$AAr?$AA?5?$AAG?$AAr?$AAo?$AAu?$AAp?$AA?$AA@ 10001158     Brackets.obj
 0001:00000190       ??_C@_1EE@CJLEEDHO@?$AAB?$AAr?$AAa?$AAc?$AAk?$AAe?$AAt?$AAs?$AA?5?$AAm?$AAa?$AAt?$AAc?$AAh?$AAi?$AAn?$AAg?$AA?5?$AAf?$AAo?$AAr?$AA?5?$AAF?$AAa?$AAr?$AA?5?$AAM?$AAa?$AAn?$AAa?$AAg?$AAe@ 10001190     Brackets.obj
 0001:000001d4       ??_C@_1BC@GJFAHMHB@?$AAB?$AAr?$AAa?$AAc?$AAk?$AAe?$AAt?$AAs?$AA?$AA@ 100011d4     Brackets.obj
 0001:000001e8       ??_C@_1BK@EKFLELHE@?$AA?1?$AA?$CK?$AA?$CK?$AA?1?$AA?$DM?$AA?$DP?$AA?$DP?$AA?$DO?$AA?$DM?$AA?$CF?$AA?$CF?$AA?$DO?$AA?$AA@ 100011e8     Brackets.obj
 0001:00000204       ??_C@_1BE@DFLFCMNK@?$AAB?$AAr?$AAa?$AAc?$AAk?$AAe?$AAt?$AAs?$AA2?$AA?$AA@ 10001204     Brackets.obj
 0001:00000218       ??_C@_1CC@FLEKOJBB@?$AA?$DM?$AA?$DO?$AA?$HL?$AA?$HN?$AA?$FL?$AA?$FN?$AA?$CI?$AA?$CJ?$AA?$CC?$AA?$CC?$AA?8?$AA?8?$AA?$CF?$AA?$CF?$AA?$KL?$AA?$LL?$AA?$AA@ 10001218     Brackets.obj
 0001:0000023c       ??_C@_1BE@CHAAIDDE@?$AAB?$AAr?$AAa?$AAc?$AAk?$AAe?$AAt?$AAs?$AA1?$AA?$AA@ 1000123c     Brackets.obj
 0001:00000250       ??_C@_1BG@KHOAFHB@?$AA?8?$AA?8?$AA?$CC?$AA?$CC?$AA?$GA?$AA?8?$AA?$GA?$AA?$GA?5?$BO?5?$BN?$AA?$AA@ 10001250     Brackets.obj
 0001:00000268       ??_C@_1BG@ICHMEPOB@?$AAQ?$AAu?$AAo?$AAt?$AAe?$AAs?$AAT?$AAy?$AAp?$AAe?$AA?$AA@ 10001268     Brackets.obj
 0001:00000280       ??_C@_19CNDHNALO@?$AAB?$AAe?$AAe?$AAp?$AA?$AA@ 10001280     Brackets.obj
 0001:0000028c       ??_C@_1BG@KDMBKMK@?$AAJ?$AAu?$AAm?$AAp?$AAT?$AAo?$AAP?$AAa?$AAi?$AAr?$AA?$AA@ 1000128c     Brackets.obj
 0001:000002a4       ??_C@_1BK@LJLNAEDP@?$AAB?$AAr?$AAa?$AAc?$AAk?$AAe?$AAt?$AAP?$AAr?$AAi?$AAo?$AAr?$AA?$AA@ 100012a4     Brackets.obj
 0001:000002c0       ??_C@_1BI@LPBIFPPH@?$AAI?$AAg?$AAn?$AAo?$AAr?$AAe?$AAA?$AAf?$AAt?$AAe?$AAr?$AA?$AA@ 100012c0     Brackets.obj
 0001:000002d8       ??_C@_1BK@LFBLPBJM@?$AAI?$AAg?$AAn?$AAo?$AAr?$AAe?$AAQ?$AAu?$AAo?$AAt?$AAe?$AAs?$AA?$AA@ 100012d8     Brackets.obj
 0001:000002f4       ??_7?$DialogItemBinding@UFarDialogItem@@@@6B@ 100012f4     Brackets.obj
 0001:000002fc       ??_7?$DialogBuilderBase@UFarDialogItem@@@@6B@ 100012fc     Brackets.obj
 0001:00000320       ??_7PluginEditFieldBinding@@6B@ 10001320     Brackets.obj
 0001:00000328       ??_7PluginDialogBuilder@@6B@ 10001328     Brackets.obj
 0001:0000034c       ??_7PluginCheckBoxBinding@@6B@ 1000134c     Brackets.obj
 0001:00000354       ??_7PluginRadioButtonBinding@@6B@ 10001354     Brackets.obj
 0001:0000035c       ??_C@_15EFLNJKHH@?$AA?$CF?$AAu?$AA?$AA@ 1000135c     Brackets.obj
 0001:00000364       ??_7PluginIntEditFieldBinding@@6B@ 10001364     Brackets.obj
 0001:0000036c       ??_7PluginUIntEditFieldBinding@@6B@ 1000136c     Brackets.obj
 0001:00000374       ??_C@_11LOCGONAA@?$AA?$AA@ 10001374     Brackets.obj
 0001:00000378       ??_C@_19MGMPFFIA@?$AAF?$AAi?$AAn?$AAd?$AA?$AA@ 10001378     Brackets.obj
 0001:00000384       ??_C@_1O@MDCABJAO@?$AAD?$AAi?$AAr?$AAe?$AAc?$AAt?$AA?$AA@ 10001384     Brackets.obj
 0001:00000394       ??_C@_1BE@LCCGEFEM@?$AAS?$AAE?$AAA?$AAR?$AAC?$AAH?$AAF?$AAW?$AAD?$AA?$AA@ 10001394     Brackets.obj
 0001:000003a8       ??_C@_1BG@LIFFHAGC@?$AAS?$AAE?$AAA?$AAR?$AAC?$AAH?$AAB?$AAA?$AAC?$AAK?$AA?$AA@ 100013a8     Brackets.obj
 0001:000003c0       ??_C@_1BE@IFIBPANP@?$AAS?$AAE?$AAL?$AAE?$AAC?$AAT?$AAF?$AAW?$AAD?$AA?$AA@ 100013c0     Brackets.obj
 0001:000003d4       ??_C@_1BG@FJDCNJBP@?$AAS?$AAE?$AAL?$AAE?$AAC?$AAT?$AAB?$AAA?$AAC?$AAK?$AA?$AA@ 100013d4     Brackets.obj
 0001:000003ec       ??_C@_1O@BAHOLLMK@?$AAC?$AAO?$AAN?$AAF?$AAI?$AAG?$AA?$AA@ 100013ec     Brackets.obj
 0001:00000400       ??_7bad_alloc@std@@6B@     10001400     LIBCMT:new.obj
 0001:00000408       ??_C@_0P@GHFPNOJB@bad?5allocation?$AA@ 10001408     LIBCMT:new.obj
 0001:00000418       __pDefaultRawDllMain       10001418     LIBCMT:dllcrt0.obj
 0001:00000418       __pRawDllMain              10001418     LIBCMT:dllcrt0.obj
 0001:00000420       ??_7exception@std@@6B@     10001420     LIBCMT:stdexcpt.obj
 0001:00000428       ??_C@_0BC@EOODALEL@Unknown?5exception?$AA@ 10001428     LIBCMT:stdexcpt.obj
 0001:00000440       ??_7type_info@@6B@         10001440     LIBCMT:typinfo.obj
 0001:00000464       ??_C@_1BK@DBDEIDLH@?$AAK?$AAE?$AAR?$AAN?$AAE?$AAL?$AA3?$AA2?$AA?4?$AAD?$AAL?$AAL?$AA?$AA@ 10001464     LIBCMT:tidtable.obj
 0001:00000480       ??_C@_07PEJMOBNF@FlsFree?$AA@ 10001480     LIBCMT:tidtable.obj
 0001:00000488       ??_C@_0M@JCPCPOEF@FlsSetValue?$AA@ 10001488     LIBCMT:tidtable.obj
 0001:00000494       ??_C@_0M@GDNOONDI@FlsGetValue?$AA@ 10001494     LIBCMT:tidtable.obj
 0001:000004a0       ??_C@_08KNHFBNJ@FlsAlloc?$AA@ 100014a0     LIBCMT:tidtable.obj
 0001:000004ac       ??_C@_0P@MIGLKIOC@CorExitProcess?$AA@ 100014ac     LIBCMT:crt0dat.obj
 0001:000004bc       ??_C@_1BI@BGOHAHKC@?$AAm?$AAs?$AAc?$AAo?$AAr?$AAe?$AAe?$AA?4?$AAd?$AAl?$AAl?$AA?$AA@ 100014bc     LIBCMT:crt0dat.obj
 0001:000004d8       __XcptActTab               100014d8     LIBCMT:winxfltr.obj
 0001:00000568       __First_FPE_Indx           10001568     LIBCMT:winxfltr.obj
 0001:0000056c       __Num_FPE                  1000156c     LIBCMT:winxfltr.obj
 0001:00000570       __XcptActTabSize           10001570     LIBCMT:winxfltr.obj
 0001:00000574       __XcptActTabCount          10001574     LIBCMT:winxfltr.obj
 0001:00000578       ??_C@_1BO@BKOMIGKJ@?$AAr?$AAu?$AAn?$AAt?$AAi?$AAm?$AAe?$AA?5?$AAe?$AAr?$AAr?$AAo?$AAr?$AA?5?$AA?$AA@ 10001578     LIBCMT:crt0msg.obj
 0001:00000598       ??_C@_15JNBOKNOG@?$AA?$AN?$AA?6?$AA?$AA@ 10001598     LIBCMT:crt0msg.obj
 0001:000005a0       ??_C@_1BM@JBBEPPHI@?$AAT?$AAL?$AAO?$AAS?$AAS?$AA?5?$AAe?$AAr?$AAr?$AAo?$AAr?$AA?$AN?$AA?6?$AA?$AA@ 100015a0     LIBCMT:crt0msg.obj
 0001:000005bc       ??_C@_1BK@KMOMNAAI@?$AAS?$AAI?$AAN?$AAG?$AA?5?$AAe?$AAr?$AAr?$AAo?$AAr?$AA?$AN?$AA?6?$AA?$AA@ 100015bc     LIBCMT:crt0msg.obj
 0001:000005d8       ??_C@_1BO@BFCDCGC@?$AAD?$AAO?$AAM?$AAA?$AAI?$AAN?$AA?5?$AAe?$AAr?$AAr?$AAo?$AAr?$AA?$AN?$AA?6?$AA?$AA@ 100015d8     LIBCMT:crt0msg.obj
 0001:000005f8       ??_C@_1BOO@KGEDBGAJ@?$AAR?$AA6?$AA0?$AA3?$AA3?$AA?$AN?$AA?6?$AA?9?$AA?5?$AAA?$AAt?$AAt?$AAe?$AAm?$AAp?$AAt?$AA?5?$AAt?$AAo?$AA?5?$AAu?$AAs?$AAe?$AA?5?$AAM?$AAS?$AAI?$AAL?$AA?5?$AAc?$AAo?$AAd@ 100015f8     LIBCMT:crt0msg.obj
 0001:000007e8       ??_C@_1GG@GOPILAJP@?$AAR?$AA6?$AA0?$AA3?$AA2?$AA?$AN?$AA?6?$AA?9?$AA?5?$AAn?$AAo?$AAt?$AA?5?$AAe?$AAn?$AAo?$AAu?$AAg?$AAh?$AA?5?$AAs?$AAp?$AAa?$AAc?$AAe?$AA?5?$AAf?$AAo?$AAr?$AA?5?$AAl?$AAo@ 100017e8     LIBCMT:crt0msg.obj
 0001:00000850       ??_C@_1MG@ENCOOIDF@?$AAR?$AA6?$AA0?$AA3?$AA1?$AA?$AN?$AA?6?$AA?9?$AA?5?$AAA?$AAt?$AAt?$AAe?$AAm?$AAp?$AAt?$AA?5?$AAt?$AAo?$AA?5?$AAi?$AAn?$AAi?$AAt?$AAi?$AAa?$AAl?$AAi?$AAz?$AAe?$AA?5?$AAt@ 10001850     LIBCMT:crt0msg.obj
 0001:00000918       ??_C@_1DO@BMFCDCD@?$AAR?$AA6?$AA0?$AA3?$AA0?$AA?$AN?$AA?6?$AA?9?$AA?5?$AAC?$AAR?$AAT?$AA?5?$AAn?$AAo?$AAt?$AA?5?$AAi?$AAn?$AAi?$AAt?$AAi?$AAa?$AAl?$AAi?$AAz?$AAe?$AAd?$AA?$AN?$AA?6?$AA?$AA@ 10001918     LIBCMT:crt0msg.obj
 0001:00000958       ??_C@_1EK@HHFLMAOL@?$AAR?$AA6?$AA0?$AA2?$AA8?$AA?$AN?$AA?6?$AA?9?$AA?5?$AAu?$AAn?$AAa?$AAb?$AAl?$AAe?$AA?5?$AAt?$AAo?$AA?5?$AAi?$AAn?$AAi?$AAt?$AAi?$AAa?$AAl?$AAi?$AAz?$AAe?$AA?5?$AAh?$AAe@ 10001958     LIBCMT:crt0msg.obj
 0001:000009a8       ??_C@_1GK@MFGOKLAG@?$AAR?$AA6?$AA0?$AA2?$AA7?$AA?$AN?$AA?6?$AA?9?$AA?5?$AAn?$AAo?$AAt?$AA?5?$AAe?$AAn?$AAo?$AAu?$AAg?$AAh?$AA?5?$AAs?$AAp?$AAa?$AAc?$AAe?$AA?5?$AAf?$AAo?$AAr?$AA?5?$AAl?$AAo@ 100019a8     LIBCMT:crt0msg.obj
 0001:00000a18       ??_C@_1GK@MCAAGJMO@?$AAR?$AA6?$AA0?$AA2?$AA6?$AA?$AN?$AA?6?$AA?9?$AA?5?$AAn?$AAo?$AAt?$AA?5?$AAe?$AAn?$AAo?$AAu?$AAg?$AAh?$AA?5?$AAs?$AAp?$AAa?$AAc?$AAe?$AA?5?$AAf?$AAo?$AAr?$AA?5?$AAs?$AAt@ 10001a18     LIBCMT:crt0msg.obj
 0001:00000a88       ??_C@_1EM@MAADIHMB@?$AAR?$AA6?$AA0?$AA2?$AA5?$AA?$AN?$AA?6?$AA?9?$AA?5?$AAp?$AAu?$AAr?$AAe?$AA?5?$AAv?$AAi?$AAr?$AAt?$AAu?$AAa?$AAl?$AA?5?$AAf?$AAu?$AAn?$AAc?$AAt?$AAi?$AAo?$AAn?$AA?5?$AAc@ 10001a88     LIBCMT:crt0msg.obj
 0001:00000ad8       ??_C@_1GK@FHCKBEFA@?$AAR?$AA6?$AA0?$AA2?$AA4?$AA?$AN?$AA?6?$AA?9?$AA?5?$AAn?$AAo?$AAt?$AA?5?$AAe?$AAn?$AAo?$AAu?$AAg?$AAh?$AA?5?$AAs?$AAp?$AAa?$AAc?$AAe?$AA?5?$AAf?$AAo?$AAr?$AA?5?$AA_?$AAo@ 10001ad8     LIBCMT:crt0msg.obj
 0001:00000b48       ??_C@_1FC@ECHBIFBC@?$AAR?$AA6?$AA0?$AA1?$AA9?$AA?$AN?$AA?6?$AA?9?$AA?5?$AAu?$AAn?$AAa?$AAb?$AAl?$AAe?$AA?5?$AAt?$AAo?$AA?5?$AAo?$AAp?$AAe?$AAn?$AA?5?$AAc?$AAo?$AAn?$AAs?$AAo?$AAl?$AAe?$AA?5@ 10001b48     LIBCMT:crt0msg.obj
 0001:00000ba0       ??_C@_1EC@JIBHAOPH@?$AAR?$AA6?$AA0?$AA1?$AA8?$AA?$AN?$AA?6?$AA?9?$AA?5?$AAu?$AAn?$AAe?$AAx?$AAp?$AAe?$AAc?$AAt?$AAe?$AAd?$AA?5?$AAh?$AAe?$AAa?$AAp?$AA?5?$AAe?$AAr?$AAr?$AAo?$AAr?$AA?$AN?$AA?6@ 10001ba0     LIBCMT:crt0msg.obj
 0001:00000be8       ??_C@_1FK@BEOGODMC@?$AAR?$AA6?$AA0?$AA1?$AA7?$AA?$AN?$AA?6?$AA?9?$AA?5?$AAu?$AAn?$AAe?$AAx?$AAp?$AAe?$AAc?$AAt?$AAe?$AAd?$AA?5?$AAm?$AAu?$AAl?$AAt?$AAi?$AAt?$AAh?$AAr?$AAe?$AAa?$AAd?$AA?5@ 10001be8     LIBCMT:crt0msg.obj
 0001:00000c48       ??_C@_1FI@LOGNIKDM@?$AAR?$AA6?$AA0?$AA1?$AA6?$AA?$AN?$AA?6?$AA?9?$AA?5?$AAn?$AAo?$AAt?$AA?5?$AAe?$AAn?$AAo?$AAu?$AAg?$AAh?$AA?5?$AAs?$AAp?$AAa?$AAc?$AAe?$AA?5?$AAf?$AAo?$AAr?$AA?5?$AAt?$AAh@ 10001c48     LIBCMT:crt0msg.obj
 0001:00000ca0       ??_C@_1EG@BEHAGFJD@?$AAR?$AA6?$AA0?$AA1?$AA0?$AA?$AN?$AA?6?$AA?9?$AA?5?$AAa?$AAb?$AAo?$AAr?$AAt?$AA?$CI?$AA?$CJ?$AA?5?$AAh?$AAa?$AAs?$AA?5?$AAb?$AAe?$AAe?$AAn?$AA?5?$AAc?$AAa?$AAl?$AAl?$AAe?$AAd@ 10001ca0     LIBCMT:crt0msg.obj
 0001:00000ce8       ??_C@_1FI@HONFMGBI@?$AAR?$AA6?$AA0?$AA0?$AA9?$AA?$AN?$AA?6?$AA?9?$AA?5?$AAn?$AAo?$AAt?$AA?5?$AAe?$AAn?$AAo?$AAu?$AAg?$AAh?$AA?5?$AAs?$AAp?$AAa?$AAc?$AAe?$AA?5?$AAf?$AAo?$AAr?$AA?5?$AAe?$AAn@ 10001ce8     LIBCMT:crt0msg.obj
 0001:00000d40       ??_C@_1FE@LLNEDJMD@?$AAR?$AA6?$AA0?$AA0?$AA8?$AA?$AN?$AA?6?$AA?9?$AA?5?$AAn?$AAo?$AAt?$AA?5?$AAe?$AAn?$AAo?$AAu?$AAg?$AAh?$AA?5?$AAs?$AAp?$AAa?$AAc?$AAe?$AA?5?$AAf?$AAo?$AAr?$AA?5?$AAa?$AAr@ 10001d40     LIBCMT:crt0msg.obj
 0001:00000d98       ??_C@_1FK@PGACCAFB@?$AAR?$AA6?$AA0?$AA0?$AA2?$AA?$AN?$AA?6?$AA?9?$AA?5?$AAf?$AAl?$AAo?$AAa?$AAt?$AAi?$AAn?$AAg?$AA?5?$AAp?$AAo?$AAi?$AAn?$AAt?$AA?5?$AAs?$AAu?$AAp?$AAp?$AAo?$AAr?$AAt?$AA?5@ 10001d98     LIBCMT:crt0msg.obj
 0001:00000ea8       ??_C@_1EK@MBDPDCGA@?$AAM?$AAi?$AAc?$AAr?$AAo?$AAs?$AAo?$AAf?$AAt?$AA?5?$AAV?$AAi?$AAs?$AAu?$AAa?$AAl?$AA?5?$AAC?$AA?$CL?$AA?$CL?$AA?5?$AAR?$AAu?$AAn?$AAt?$AAi?$AAm?$AAe?$AA?5?$AAL?$AAi?$AAb@ 10001ea8     LIBCMT:crt0msg.obj
 0001:00000ef4       ??_C@_15IABLJNFO@?$AA?6?$AA?6?$AA?$AA@ 10001ef4     LIBCMT:crt0msg.obj
 0001:00000efc       ??_C@_17LGKOMLJ@?$AA?4?$AA?4?$AA?4?$AA?$AA@ 10001efc     LIBCMT:crt0msg.obj
 0001:00000f04       ??_C@_1CO@EAEJAADC@?$AA?$DM?$AAp?$AAr?$AAo?$AAg?$AAr?$AAa?$AAm?$AA?5?$AAn?$AAa?$AAm?$AAe?$AA?5?$AAu?$AAn?$AAk?$AAn?$AAo?$AAw?$AAn?$AA?$DO?$AA?$AA@ 10001f04     LIBCMT:crt0msg.obj
 0001:00000f34       ??_C@_1DE@JNGNBFGO@?$AAR?$AAu?$AAn?$AAt?$AAi?$AAm?$AAe?$AA?5?$AAE?$AAr?$AAr?$AAo?$AAr?$AA?$CB?$AA?6?$AA?6?$AAP?$AAr?$AAo?$AAg?$AAr?$AAa?$AAm?$AA?3?$AA?5?$AA?$AA@ 10001f34     LIBCMT:crt0msg.obj
 0001:00000f68       ??_C@_1BC@GDGBMEMK@?$AAH?$AAH?$AA?3?$AAm?$AAm?$AA?3?$AAs?$AAs?$AA?$AA@ 10001f68     LIBCMT:nlsdata2.obj
 0001:00000f7c       ??_C@_1CI@KNAKOEBC@?$AAd?$AAd?$AAd?$AAd?$AA?0?$AA?5?$AAM?$AAM?$AAM?$AAM?$AA?5?$AAd?$AAd?$AA?0?$AA?5?$AAy?$AAy?$AAy?$AAy?$AA?$AA@ 10001f7c     LIBCMT:nlsdata2.obj
 0001:00000fa4       ??_C@_1BC@IEBCMHCM@?$AAM?$AAM?$AA?1?$AAd?$AAd?$AA?1?$AAy?$AAy?$AA?$AA@ 10001fa4     LIBCMT:nlsdata2.obj
 0001:00000fb8       ??_C@_15CLMNNGEL@?$AAP?$AAM?$AA?$AA@ 10001fb8     LIBCMT:nlsdata2.obj
 0001:00000fc0       ??_C@_15ODEHAHHF@?$AAA?$AAM?$AA?$AA@ 10001fc0     LIBCMT:nlsdata2.obj
 0001:00000fc8       ??_C@_1BC@FEMKIFH@?$AAD?$AAe?$AAc?$AAe?$AAm?$AAb?$AAe?$AAr?$AA?$AA@ 10001fc8     LIBCMT:nlsdata2.obj
 0001:00000fdc       ??_C@_1BC@BGLIFPF@?$AAN?$AAo?$AAv?$AAe?$AAm?$AAb?$AAe?$AAr?$AA?$AA@ 10001fdc     LIBCMT:nlsdata2.obj
 0001:00000ff0       ??_C@_1BA@EPANDLNG@?$AAO?$AAc?$AAt?$AAo?$AAb?$AAe?$AAr?$AA?$AA@ 10001ff0     LIBCMT:nlsdata2.obj
 0001:00001000       ??_C@_1BE@DKAAMBJL@?$AAS?$AAe?$AAp?$AAt?$AAe?$AAm?$AAb?$AAe?$AAr?$AA?$AA@ 10002000     LIBCMT:nlsdata2.obj
 0001:00001014       ??_C@_1O@PAHLKOAC@?$AAA?$AAu?$AAg?$AAu?$AAs?$AAt?$AA?$AA@ 10002014     LIBCMT:nlsdata2.obj
 0001:00001024       ??_C@_19BIFMLPCD@?$AAJ?$AAu?$AAl?$AAy?$AA?$AA@ 10002024     LIBCMT:nlsdata2.obj
 0001:00001030       ??_C@_19EPFLPGAP@?$AAJ?$AAu?$AAn?$AAe?$AA?$AA@ 10002030     LIBCMT:nlsdata2.obj
 0001:0000103c       ??_C@_1M@GJNLMHFD@?$AAA?$AAp?$AAr?$AAi?$AAl?$AA?$AA@ 1000203c     LIBCMT:nlsdata2.obj
 0001:00001048       ??_C@_1M@IKEENEDF@?$AAM?$AAa?$AAr?$AAc?$AAh?$AA?$AA@ 10002048     LIBCMT:nlsdata2.obj
 0001:00001054       ??_C@_1BC@JGDDFFAM@?$AAF?$AAe?$AAb?$AAr?$AAu?$AAa?$AAr?$AAy?$AA?$AA@ 10002054     LIBCMT:nlsdata2.obj
 0001:00001068       ??_C@_1BA@EFMEIEBA@?$AAJ?$AAa?$AAn?$AAu?$AAa?$AAr?$AAy?$AA?$AA@ 10002068     LIBCMT:nlsdata2.obj
 0001:00001078       ??_C@_17EGKACKIF@?$AAD?$AAe?$AAc?$AA?$AA@ 10002078     LIBCMT:nlsdata2.obj
 0001:00001080       ??_C@_17BBDMLCIG@?$AAN?$AAo?$AAv?$AA?$AA@ 10002080     LIBCMT:nlsdata2.obj
 0001:00001088       ??_C@_17FNLKOI@?$AAO?$AAc?$AAt?$AA?$AA@ 10002088     LIBCMT:nlsdata2.obj
 0001:00001090       ??_C@_17HCHCOKMG@?$AAS?$AAe?$AAp?$AA?$AA@ 10002090     LIBCMT:nlsdata2.obj
 0001:00001098       ??_C@_17ICPELBCN@?$AAA?$AAu?$AAg?$AA?$AA@ 10002098     LIBCMT:nlsdata2.obj
 0001:000010a0       ??_C@_17IJPCKHK@?$AAJ?$AAu?$AAl?$AA?$AA@ 100020a0     LIBCMT:nlsdata2.obj
 0001:000010a8       ??_C@_17KCJGOCPB@?$AAJ?$AAu?$AAn?$AA?$AA@ 100020a8     LIBCMT:nlsdata2.obj
 0001:000010b0       ??_C@_17PNNKMEED@?$AAM?$AAa?$AAy?$AA?$AA@ 100020b0     LIBCMT:nlsdata2.obj
 0001:000010b8       ??_C@_17LFPOIHDD@?$AAA?$AAp?$AAr?$AA?$AA@ 100020b8     LIBCMT:nlsdata2.obj
 0001:000010c0       ??_C@_17CKNLEDEC@?$AAM?$AAa?$AAr?$AA?$AA@ 100020c0     LIBCMT:nlsdata2.obj
 0001:000010c8       ??_C@_17LMDJEKJN@?$AAF?$AAe?$AAb?$AA?$AA@ 100020c8     LIBCMT:nlsdata2.obj
 0001:000010d0       ??_C@_17DKNBKCHM@?$AAJ?$AAa?$AAn?$AA?$AA@ 100020d0     LIBCMT:nlsdata2.obj
 0001:000010d8       ??_C@_1BC@ENMNNPAJ@?$AAS?$AAa?$AAt?$AAu?$AAr?$AAd?$AAa?$AAy?$AA?$AA@ 100020d8     LIBCMT:nlsdata2.obj
 0001:000010ec       ??_C@_1O@PDICJHAG@?$AAF?$AAr?$AAi?$AAd?$AAa?$AAy?$AA?$AA@ 100020ec     LIBCMT:nlsdata2.obj
 0001:000010fc       ??_C@_1BC@HHMNLIHE@?$AAT?$AAh?$AAu?$AAr?$AAs?$AAd?$AAa?$AAy?$AA?$AA@ 100020fc     LIBCMT:nlsdata2.obj
 0001:00001110       ??_C@_1BE@EBOGMDOH@?$AAW?$AAe?$AAd?$AAn?$AAe?$AAs?$AAd?$AAa?$AAy?$AA?$AA@ 10002110     LIBCMT:nlsdata2.obj
 0001:00001124       ??_C@_1BA@ENFBFFEK@?$AAT?$AAu?$AAe?$AAs?$AAd?$AAa?$AAy?$AA?$AA@ 10002124     LIBCMT:nlsdata2.obj
 0001:00001134       ??_C@_1O@MMNBFLIA@?$AAM?$AAo?$AAn?$AAd?$AAa?$AAy?$AA?$AA@ 10002134     LIBCMT:nlsdata2.obj
 0001:00001144       ??_C@_1O@IHNHDHPB@?$AAS?$AAu?$AAn?$AAd?$AAa?$AAy?$AA?$AA@ 10002144     LIBCMT:nlsdata2.obj
 0001:00001154       ??_C@_17GGIBDPIH@?$AAS?$AAa?$AAt?$AA?$AA@ 10002154     LIBCMT:nlsdata2.obj
 0001:0000115c       ??_C@_17HFOLPPLP@?$AAF?$AAr?$AAi?$AA?$AA@ 1000215c     LIBCMT:nlsdata2.obj
 0001:00001164       ??_C@_17PDPHAADD@?$AAT?$AAh?$AAu?$AA?$AA@ 10002164     LIBCMT:nlsdata2.obj
 0001:0000116c       ??_C@_17CJEDCEPE@?$AAW?$AAe?$AAd?$AA?$AA@ 1000216c     LIBCMT:nlsdata2.obj
 0001:00001174       ??_C@_17BMKGEGOJ@?$AAT?$AAu?$AAe?$AA?$AA@ 10002174     LIBCMT:nlsdata2.obj
 0001:0000117c       ??_C@_17KBOMKBF@?$AAM?$AAo?$AAn?$AA?$AA@ 1000217c     LIBCMT:nlsdata2.obj
 0001:00001184       ??_C@_17MBGCMIPB@?$AAS?$AAu?$AAn?$AA?$AA@ 10002184     LIBCMT:nlsdata2.obj
 0001:0000118c       ??_C@_08JCCMCCIL@HH?3mm?3ss?$AA@ 1000218c     LIBCMT:nlsdata2.obj
 0001:00001198       ??_C@_0BE@CKGJFCPC@dddd?0?5MMMM?5dd?0?5yyyy?$AA@ 10002198     LIBCMT:nlsdata2.obj
 0001:000011ac       ??_C@_08BPBNCDIB@MM?1dd?1yy?$AA@ 100021ac     LIBCMT:nlsdata2.obj
 0001:000011b8       ??_C@_02CJNFDJBF@PM?$AA@   100021b8     LIBCMT:nlsdata2.obj
 0001:000011bc       ??_C@_02DEDBPAFC@AM?$AA@   100021bc     LIBCMT:nlsdata2.obj
 0001:000011c0       ??_C@_08EDHMEBNP@December?$AA@ 100021c0     LIBCMT:nlsdata2.obj
 0001:000011cc       ??_C@_08HCHEGEOA@November?$AA@ 100021cc     LIBCMT:nlsdata2.obj
 0001:000011d8       ??_C@_07JJNFCEND@October?$AA@ 100021d8     LIBCMT:nlsdata2.obj
 0001:000011e0       ??_C@_09BHHEALKD@September?$AA@ 100021e0     LIBCMT:nlsdata2.obj
 0001:000011ec       ??_C@_06LBBHFDDG@August?$AA@ 100021ec     LIBCMT:nlsdata2.obj
 0001:000011f4       ??_C@_04MIEPOIFP@July?$AA@ 100021f4     LIBCMT:nlsdata2.obj
 0001:000011fc       ??_C@_04CNLMGBGM@June?$AA@ 100021fc     LIBCMT:nlsdata2.obj
 0001:00001204       ??_C@_05DMJDNLEJ@April?$AA@ 10002204     LIBCMT:nlsdata2.obj
 0001:0000120c       ??_C@_05HPCKOFNC@March?$AA@ 1000220c     LIBCMT:nlsdata2.obj
 0001:00001214       ??_C@_08GNJGEPFN@February?$AA@ 10002214     LIBCMT:nlsdata2.obj
 0001:00001220       ??_C@_07CGJPFGJA@January?$AA@ 10002220     LIBCMT:nlsdata2.obj
 0001:00001228       ??_C@_03MKABNOCG@Dec?$AA@  10002228     LIBCMT:nlsdata2.obj
 0001:0000122c       ??_C@_03JPJOFNIA@Nov?$AA@  1000222c     LIBCMT:nlsdata2.obj
 0001:00001230       ??_C@_03BMAOKBAD@Oct?$AA@  10002230     LIBCMT:nlsdata2.obj
 0001:00001234       ??_C@_03GGCAPAJC@Sep?$AA@  10002234     LIBCMT:nlsdata2.obj
 0001:00001238       ??_C@_03IFJFEIGA@Aug?$AA@  10002238     LIBCMT:nlsdata2.obj
 0001:0000123c       ??_C@_03LBGABGKK@Jul?$AA@  1000223c     LIBCMT:nlsdata2.obj
 0001:00001240       ??_C@_03IDFGHECI@Jun?$AA@  10002240     LIBCMT:nlsdata2.obj
 0001:00001244       ??_C@_03CNMDKL@May?$AA@    10002244     LIBCMT:nlsdata2.obj
 0001:00001248       ??_C@_03LEOLGMJP@Apr?$AA@  10002248     LIBCMT:nlsdata2.obj
 0001:0000124c       ??_C@_03ODNJBKGA@Mar?$AA@  1000224c     LIBCMT:nlsdata2.obj
 0001:00001250       ??_C@_03HJBDCHOM@Feb?$AA@  10002250     LIBCMT:nlsdata2.obj
 0001:00001254       ??_C@_03JIHJHPIE@Jan?$AA@  10002254     LIBCMT:nlsdata2.obj
 0001:00001258       ??_C@_08INBOOONO@Saturday?$AA@ 10002258     LIBCMT:nlsdata2.obj
 0001:00001264       ??_C@_06JECMNKMI@Friday?$AA@ 10002264     LIBCMT:nlsdata2.obj
 0001:0000126c       ??_C@_08HACCIKIA@Thursday?$AA@ 1000226c     LIBCMT:nlsdata2.obj
 0001:00001278       ??_C@_09DLIGFAKA@Wednesday?$AA@ 10002278     LIBCMT:nlsdata2.obj
 0001:00001284       ??_C@_07BAAGCFCM@Tuesday?$AA@ 10002284     LIBCMT:nlsdata2.obj
 0001:0000128c       ??_C@_06JLEDEDGH@Monday?$AA@ 1000228c     LIBCMT:nlsdata2.obj
 0001:00001294       ??_C@_06OOPIFAJ@Sunday?$AA@ 10002294     LIBCMT:nlsdata2.obj
 0001:0000129c       ??_C@_03FEFJNEK@Sat?$AA@   1000229c     LIBCMT:nlsdata2.obj
 0001:000012a0       ??_C@_03IDIOELNC@Fri?$AA@  100022a0     LIBCMT:nlsdata2.obj
 0001:000012a4       ??_C@_03IOFIKPDN@Thu?$AA@  100022a4     LIBCMT:nlsdata2.obj
 0001:000012a8       ??_C@_03MHOMLAJA@Wed?$AA@  100022a8     LIBCMT:nlsdata2.obj
 0001:000012ac       ??_C@_03NAGEINEP@Tue?$AA@  100022ac     LIBCMT:nlsdata2.obj
 0001:000012b0       ??_C@_03PDAGKDH@Mon?$AA@   100022b0     LIBCMT:nlsdata2.obj
 0001:000012b4       ??_C@_03KOEHGMDN@Sun?$AA@  100022b4     LIBCMT:nlsdata2.obj
 0001:000012b8       ??_C@_0BK@CFCOFLF@?5Complete?5Object?5Locator?8?$AA@ 100022b8     LIBCMT:undname.obj
 0001:000012d4       ??_C@_0BN@MECKDCOJ@?5Class?5Hierarchy?5Descriptor?8?$AA@ 100022d4     LIBCMT:undname.obj
 0001:000012f4       ??_C@_0BD@LGICGFMM@?5Base?5Class?5Array?8?$AA@ 100022f4     LIBCMT:undname.obj
 0001:00001308       ??_C@_0BM@LDKODKLH@?5Base?5Class?5Descriptor?5at?5?$CI?$AA@ 10002308     LIBCMT:undname.obj
 0001:00001324       ??_C@_0BC@DAFEJGAK@?5Type?5Descriptor?8?$AA@ 10002324     LIBCMT:undname.obj
 0001:00001338       ??_C@_0BM@PMGGMLDN@?$GAlocal?5static?5thread?5guard?8?$AA@ 10002338     LIBCMT:undname.obj
 0001:00001354       ??_C@_0CL@FGIJHLCE@?$GAmanaged?5vector?5copy?5constructor@ 10002354     LIBCMT:undname.obj
 0001:00001380       ??_C@_0CJ@GJELGAMM@?$GAvector?5vbase?5copy?5constructor?5i@ 10002380     LIBCMT:undname.obj
 0001:000013ac       ??_C@_0CD@CGAJBKEJ@?$GAvector?5copy?5constructor?5iterato@ 100023ac     LIBCMT:undname.obj
 0001:000013d0       ??_C@_0CB@PDBIFEP@?$GAdynamic?5atexit?5destructor?5for?5?8@ 100023d0     LIBCMT:undname.obj
 0001:000013f4       ??_C@_0BL@CLIPGLGB@?$GAdynamic?5initializer?5for?5?8?$AA@ 100023f4     LIBCMT:undname.obj
 0001:00001410       ??_C@_0CM@FCBBDIGB@?$GAeh?5vector?5vbase?5copy?5constructo@ 10002410     LIBCMT:undname.obj
 0001:0000143c       ??_C@_0CG@HLDDJMAG@?$GAeh?5vector?5copy?5constructor?5iter@ 1000243c     LIBCMT:undname.obj
 0001:00001464       ??_C@_0CF@IMGKMJNO@?$GAmanaged?5vector?5destructor?5itera@ 10002464     LIBCMT:undname.obj
 0001:0000148c       ??_C@_0CG@CFDHKGGD@?$GAmanaged?5vector?5constructor?5iter@ 1000248c     LIBCMT:undname.obj
 0001:000014b4       ??_C@_0BN@CKNJLHMB@?$GAplacement?5delete?$FL?$FN?5closure?8?$AA@ 100024b4     LIBCMT:undname.obj
 0001:000014d4       ??_C@_0BL@CNOONJFP@?$GAplacement?5delete?5closure?8?$AA@ 100024d4     LIBCMT:undname.obj
 0001:000014f0       ??_C@_0P@HJKNJFNN@?$GAomni?5callsig?8?$AA@ 100024f0     LIBCMT:undname.obj
 0001:00001500       ??_C@_09LBNFPBCA@?5delete?$FL?$FN?$AA@ 10002500     LIBCMT:undname.obj
 0001:0000150c       ??_C@_06FHBGPFGH@?5new?$FL?$FN?$AA@ 1000250c     LIBCMT:undname.obj
 0001:00001514       ??_C@_0CE@IIHCMGGL@?$GAlocal?5vftable?5constructor?5closu@ 10002514     LIBCMT:undname.obj
 0001:00001538       ??_C@_0BA@KKLDJDLB@?$GAlocal?5vftable?8?$AA@ 10002538     LIBCMT:undname.obj
 0001:00001548       ??_C@_05KHLCHHI@?$GARTTI?$AA@ 10002548     LIBCMT:undname.obj
 0001:00001550       ??_C@_03KLGMFNMG@?$GAEH?$AA@ 10002550     LIBCMT:undname.obj
 0001:00001554       ??_C@_0BA@KBCDOMBN@?$GAudt?5returning?8?$AA@ 10002554     LIBCMT:undname.obj
 0001:00001564       ??_C@_0BL@LLKPOHJI@?$GAcopy?5constructor?5closure?8?$AA@ 10002564     LIBCMT:undname.obj
 0001:00001580       ??_C@_0CH@OOJPLCPH@?$GAeh?5vector?5vbase?5constructor?5ite@ 10002580     LIBCMT:undname.obj
 0001:000015a8       ??_C@_0CA@GCEOPDGL@?$GAeh?5vector?5destructor?5iterator?8?$AA@ 100025a8     LIBCMT:undname.obj
 0001:000015c8       ??_C@_0CB@JONCMFFK@?$GAeh?5vector?5constructor?5iterator?8@ 100025c8     LIBCMT:undname.obj
 0001:000015ec       ??_C@_0BL@NILFHHPC@?$GAvirtual?5displacement?5map?8?$AA@ 100025ec     LIBCMT:undname.obj
 0001:00001608       ??_C@_0CE@IKBNEHA@?$GAvector?5vbase?5constructor?5iterat@ 10002608     LIBCMT:undname.obj
 0001:0000162c       ??_C@_0BN@LFPFMEDL@?$GAvector?5destructor?5iterator?8?$AA@ 1000262c     LIBCMT:undname.obj
 0001:0000164c       ??_C@_0BO@PFGOCPJJ@?$GAvector?5constructor?5iterator?8?$AA@ 1000264c     LIBCMT:undname.obj
 0001:0000166c       ??_C@_0BN@IMDCHIKM@?$GAscalar?5deleting?5destructor?8?$AA@ 1000266c     LIBCMT:undname.obj
 0001:0000168c       ??_C@_0BO@OBMKPJIG@?$GAdefault?5constructor?5closure?8?$AA@ 1000268c     LIBCMT:undname.obj
 0001:000016ac       ??_C@_0BN@DEGPLNFK@?$GAvector?5deleting?5destructor?8?$AA@ 100026ac     LIBCMT:undname.obj
 0001:000016cc       ??_C@_0BD@JDLKDPAB@?$GAvbase?5destructor?8?$AA@ 100026cc     LIBCMT:undname.obj
 0001:000016e0       ??_C@_08OBABFOLI@?$GAstring?8?$AA@ 100026e0     LIBCMT:undname.obj
 0001:000016ec       ??_C@_0BF@KDPPACIK@?$GAlocal?5static?5guard?8?$AA@ 100026ec     LIBCMT:undname.obj
 0001:00001704       ??_C@_08LLFFHHDJ@?$GAtypeof?8?$AA@ 10002704     LIBCMT:undname.obj
 0001:00001710       ??_C@_07FEEIOKP@?$GAvcall?8?$AA@ 10002710     LIBCMT:undname.obj
 0001:00001718       ??_C@_09BLBHBJP@?$GAvbtable?8?$AA@ 10002718     LIBCMT:undname.obj
 0001:00001724       ??_C@_09IFPLHPGF@?$GAvftable?8?$AA@ 10002724     LIBCMT:undname.obj
 0001:00001730       ??_C@_02MHEGNOJ@?$FO?$DN?$AA@ 10002730     LIBCMT:undname.obj
 0001:00001734       ??_C@_02DHLNPPGH@?$HM?$DN?$AA@ 10002734     LIBCMT:undname.obj
 0001:00001738       ??_C@_02FGJGFEAB@?$CG?$DN?$AA@ 10002738     LIBCMT:undname.obj
 0001:0000173c       ??_C@_03CDNPDDLA@?$DM?$DM?$DN?$AA@ 1000273c     LIBCMT:undname.obj
 0001:00001740       ??_C@_03IKFCCPFF@?$DO?$DO?$DN?$AA@ 10002740     LIBCMT:undname.obj
 0001:00001744       ??_C@_02FENAOKFI@?$CF?$DN?$AA@ 10002744     LIBCMT:undname.obj
 0001:00001748       ??_C@_02FJEHGPIO@?1?$DN?$AA@ 10002748     LIBCMT:undname.obj
 0001:0000174c       ??_C@_02FKMDLLOA@?9?$DN?$AA@ 1000274c     LIBCMT:undname.obj
 0001:00001750       ??_C@_02FOEOMHFC@?$CL?$DN?$AA@ 10002750     LIBCMT:undname.obj
 0001:00001754       ??_C@_02FPIMKNGF@?$CK?$DN?$AA@ 10002754     LIBCMT:undname.obj
 0001:00001758       ??_C@_02NONPIBCD@?$HM?$HM?$AA@ 10002758     LIBCMT:undname.obj
 0001:0000175c       ??_C@_02PPKAJPJL@?$CG?$CG?$AA@ 1000275c     LIBCMT:undname.obj
 0001:00001760       ??_C@_01DNKMNLPK@?$HM?$AA@ 10002760     LIBCMT:undname.obj
 0001:00001764       ??_C@_01JKBOJNNK@?$FO?$AA@ 10002764     LIBCMT:undname.obj
 0001:00001768       ??_C@_01PJKLJHI@?$HO?$AA@  10002768     LIBCMT:undname.obj
 0001:0000176c       ??_C@_02HCKGKOFO@?$CI?$CJ?$AA@ 1000276c     LIBCMT:undname.obj
 0001:00001770       ??_C@_01IHBHIGKO@?0?$AA@   10002770     LIBCMT:undname.obj
 0001:00001774       ??_C@_02EEKDKGMJ@?$DO?$DN?$AA@ 10002774     LIBCMT:undname.obj
 0001:00001778       ??_C@_01PPODPGHN@?$DO?$AA@ 10002778     LIBCMT:undname.obj
 0001:0000177c       ??_C@_02EHCHHCKH@?$DM?$DN?$AA@ 1000277c     LIBCMT:undname.obj
 0001:00001780       ??_C@_01MNNFJEPP@?$DM?$AA@ 10002780     LIBCMT:undname.obj
 0001:00001784       ??_C@_01FGNFDNOH@?$CF?$AA@ 10002784     LIBCMT:undname.obj
 0001:00001788       ??_C@_01KMDKNFGN@?1?$AA@   10002788     LIBCMT:undname.obj
 0001:0000178c       ??_C@_03MNHNFDLC@?9?$DO?$CK?$AA@ 1000278c     LIBCMT:undname.obj
 0001:00001790       ??_C@_01HNPIGOCE@?$CG?$AA@ 10002790     LIBCMT:undname.obj
 0001:00001794       ??_C@_01MIFGBAGJ@?$CL?$AA@ 10002794     LIBCMT:undname.obj
 0001:00001798       ??_C@_01JOAMLHOP@?9?$AA@   10002798     LIBCMT:undname.obj
 0001:0000179c       ??_C@_02BAABKJLB@?9?9?$AA@ 1000279c     LIBCMT:undname.obj
 0001:000017a0       ??_C@_02ECNGHCIF@?$CL?$CL?$AA@ 100027a0     LIBCMT:undname.obj
 0001:000017a4       ??_C@_01NBENCBCI@?$CK?$AA@ 100027a4     LIBCMT:undname.obj
 0001:000017a8       ??_C@_02HBOOOICD@?9?$DO?$AA@ 100027a8     LIBCMT:undname.obj
 0001:000017ac       ??_C@_08LHJFAFGD@operator?$AA@ 100027ac     LIBCMT:undname.obj
 0001:000017b8       ??_C@_02GPECMEKF@?$FL?$FN?$AA@ 100027b8     LIBCMT:undname.obj
 0001:000017bc       ??_C@_02FDNJECIE@?$CB?$DN?$AA@ 100027bc     LIBCMT:undname.obj
 0001:000017c0       ??_C@_02EGOFBIJA@?$DN?$DN?$AA@ 100027c0     LIBCMT:undname.obj
 0001:000017c4       ??_C@_01DCLJPIOD@?$CB?$AA@ 100027c4     LIBCMT:undname.obj
 0001:000017c8       ??_C@_02FODMEDOG@?$DM?$DM?$AA@ 100027c8     LIBCMT:undname.obj
 0001:000017cc       ??_C@_02GPIOPFAK@?$DO?$DO?$AA@ 100027cc     LIBCMT:undname.obj
 0001:000017d0       ??_C@_01NEMOKFLO@?$DN?$AA@ 100027d0     LIBCMT:undname.obj
 0001:000017d4       ??_C@_07FPCDHGMM@?5delete?$AA@ 100027d4     LIBCMT:undname.obj
 0001:000017dc       ??_C@_04NIHEBCM@?5new?$AA@ 100027dc     LIBCMT:undname.obj
 0001:000017e1       ??_C@_00CNPNBAHC@?$AA@     100027e1     LIBCMT:undname.obj
 0001:000017e4       ??_C@_0M@GFIIJFMG@__unaligned?$AA@ 100027e4     LIBCMT:undname.obj
 0001:000017f0       ??_C@_0L@PILCLIHE@__restrict?$AA@ 100027f0     LIBCMT:undname.obj
 0001:000017fc       ??_C@_07JOMMBBKO@__ptr64?$AA@ 100027fc     LIBCMT:undname.obj
 0001:00001804       ??_C@_06GHPCKEAG@__eabi?$AA@ 10002804     LIBCMT:undname.obj
 0001:0000180c       ??_C@_09HIJEGCPM@__clrcall?$AA@ 1000280c     LIBCMT:undname.obj
 0001:00001818       ??_C@_0L@JMKHOMEK@__fastcall?$AA@ 10002818     LIBCMT:undname.obj
 0001:00001824       ??_C@_0L@NPHFGOKO@__thiscall?$AA@ 10002824     LIBCMT:undname.obj
 0001:00001830       ??_C@_09IFJBGAPI@__stdcall?$AA@ 10002830     LIBCMT:undname.obj
 0001:0000183c       ??_C@_08GHMPAG@__pascal?$AA@ 1000283c     LIBCMT:undname.obj
 0001:00001848       ??_C@_07KOLFKCDI@__cdecl?$AA@ 10002848     LIBCMT:undname.obj
 0001:00001850       ??_C@_08EHJDFFNH@__based?$CI?$AA@ 10002850     LIBCMT:undname.obj
 0001:000019e4       ??_C@_0BI@DFKBFLJE@GetProcessWindowStation?$AA@ 100029e4     LIBCMT:crtmboxw.obj
 0001:000019fc       ??_C@_0BK@DEKFELLI@GetUserObjectInformationW?$AA@ 100029fc     LIBCMT:crtmboxw.obj
 0001:00001a18       ??_C@_0BD@HHGDFDBJ@GetLastActivePopup?$AA@ 10002a18     LIBCMT:crtmboxw.obj
 0001:00001a2c       ??_C@_0BA@HNOPNCHB@GetActiveWindow?$AA@ 10002a2c     LIBCMT:crtmboxw.obj
 0001:00001a3c       ??_C@_0M@DLDCCGNP@MessageBoxW?$AA@ 10002a3c     LIBCMT:crtmboxw.obj
 0001:00001a48       ??_C@_1BG@GOEBHBDC@?$AAU?$AAS?$AAE?$AAR?$AA3?$AA2?$AA?4?$AAD?$AAL?$AAL?$AA?$AA@ 10002a48     LIBCMT:crtmboxw.obj
 0001:00001a60       ___newctype                10002a60     LIBCMT:ctype.obj
 0001:00001d60       __wctype                   10002d60     LIBCMT:ctype.obj
 0001:00001f68       ___newclmap                10002f68     LIBCMT:ctype.obj
 0001:000020e8       ___newcumap                100030e8     LIBCMT:ctype.obj
 0001:000022f0       __load_config_used         100032f0     LIBCMT:loadcfg.obj
 0001:00002338       ??_R4bad_alloc@std@@6B@    10003338     LIBCMT:new.obj
 0001:0000234c       ??_R3bad_alloc@std@@8      1000334c     LIBCMT:new.obj
 0001:0000235c       ??_R2bad_alloc@std@@8      1000335c     LIBCMT:new.obj
 0001:00002368       ??_R1A@?0A@EA@bad_alloc@std@@8 10003368     LIBCMT:new.obj
 0001:00002384       ??_R1A@?0A@EA@exception@std@@8 10003384     LIBCMT:new.obj
 0001:000023a0       ??_R3exception@std@@8      100033a0     LIBCMT:new.obj
 0001:000023b0       ??_R2exception@std@@8      100033b0     LIBCMT:new.obj
 0001:000023b8       ??_R4exception@std@@6B@    100033b8     LIBCMT:stdexcpt.obj
 0001:000023cc       ??_R4type_info@@6B@        100033cc     LIBCMT:typinfo.obj
 0001:000023e0       ??_R3type_info@@8          100033e0     LIBCMT:typinfo.obj
 0001:000023f0       ??_R2type_info@@8          100033f0     LIBCMT:typinfo.obj
 0001:000023f8       ??_R1A@?0A@EA@type_info@@8 100033f8     LIBCMT:typinfo.obj
 0001:00002420       ___safe_se_handler_table   10003420     <linker-defined>
 0001:0000242c       ___rtc_iaa                 1000342c     LIBCMT:_initsect_.obj
 0001:00002430       ___rtc_izz                 10003430     LIBCMT:_initsect_.obj
 0001:00002434       ___rtc_taa                 10003434     LIBCMT:_initsect_.obj
 0001:00002438       ___rtc_tzz                 10003438     LIBCMT:_initsect_.obj
 0001:00002440       __alloca_probe             10003440     chkstk.obj
 0001:00002440       __chkstk                   10003440 f   chkstk.obj
 0001:00002470       ?GetLangString@PluginDialogBuilder@@MAEPB_WH@Z 10003470 f i Brackets.obj
 0001:00002490       _GetGlobalInfoW@4          10003490 f   Brackets.obj
 0001:00002510       _SetStartupInfoW@4         10003510 f   Brackets.obj
 0001:000027e0       _GetPluginInfoW@4          100037e0 f   Brackets.obj
 0001:00002830       ?SaveValue@?$DialogItemBinding@UFarDialogItem@@@@UAEXPAUFarDialogItem@@H@Z 10003830 f i Brackets.obj
 0001:00002830       ?InitDialogItem@?$DialogBuilderBase@UFarDialogItem@@@@MAEXPAUFarDialogItem@@PB_W@Z 10003830 f i Brackets.obj
 0001:00002840       ?TextWidth@?$DialogBuilderBase@UFarDialogItem@@@@MAEHABUFarDialogItem@@@Z 10003840 f i Brackets.obj
 0001:00002850       ?DoShowDialog@?$DialogBuilderBase@UFarDialogItem@@@@MAEHXZ 10003850 f i Brackets.obj
 0001:00002860       ?CreateRadioButtonBinding@?$DialogBuilderBase@UFarDialogItem@@@@MAEPAU?$DialogItemBinding@UFarDialogItem@@@@PAH@Z 10003860 f i Brackets.obj
 0001:00002860       ?GetLangString@?$DialogBuilderBase@UFarDialogItem@@@@MAEPB_WH@Z 10003860 f i Brackets.obj
 0001:00002870       ??1?$DialogBuilderBase@UFarDialogItem@@@@MAE@XZ 10003870 f i Brackets.obj
 0001:000028c0       ?CreateCheckBoxBinding@?$DialogBuilderBase@UFarDialogItem@@@@MAEPAU?$DialogItemBinding@UFarDialogItem@@@@PAHH@Z 100038c0 f i Brackets.obj
 0001:000028c0       ?AddIntEditField@?$DialogBuilderBase@UFarDialogItem@@@@UAEPAUFarDialogItem@@PAHH@Z 100038c0 f i Brackets.obj
 0001:000028c0       ?AddUIntEditField@?$DialogBuilderBase@UFarDialogItem@@@@UAEPAUFarDialogItem@@PAIH@Z 100038c0 f i Brackets.obj
 0001:000028d0       ??_EPluginUIntEditFieldBinding@@UAEPAXI@Z 100038d0 f i Brackets.obj
 0001:000028d0       ??_GPluginUIntEditFieldBinding@@UAEPAXI@Z 100038d0 f i Brackets.obj
 0001:000028d0       ??_GPluginEditFieldBinding@@UAEPAXI@Z 100038d0 f i Brackets.obj
 0001:000028d0       ??_GPluginCheckBoxBinding@@UAEPAXI@Z 100038d0 f i Brackets.obj
 0001:000028d0       ??_EPluginIntEditFieldBinding@@UAEPAXI@Z 100038d0 f i Brackets.obj
 0001:000028d0       ??_GPluginRadioButtonBinding@@UAEPAXI@Z 100038d0 f i Brackets.obj
 0001:000028d0       ??_G?$DialogItemBinding@UFarDialogItem@@@@UAEPAXI@Z 100038d0 f i Brackets.obj
 0001:000028d0       ??_E?$DialogItemBinding@UFarDialogItem@@@@UAEPAXI@Z 100038d0 f i Brackets.obj
 0001:000028d0       ??_EPluginEditFieldBinding@@UAEPAXI@Z 100038d0 f i Brackets.obj
 0001:000028d0       ??_GPluginIntEditFieldBinding@@UAEPAXI@Z 100038d0 f i Brackets.obj
 0001:000028d0       ??_EPluginRadioButtonBinding@@UAEPAXI@Z 100038d0 f i Brackets.obj
 0001:000028d0       ??_EPluginCheckBoxBinding@@UAEPAXI@Z 100038d0 f i Brackets.obj
 0001:000028f0       ??_G?$DialogBuilderBase@UFarDialogItem@@@@MAEPAXI@Z 100038f0 f i Brackets.obj
 0001:000028f0       ??_E?$DialogBuilderBase@UFarDialogItem@@@@MAEPAXI@Z 100038f0 f i Brackets.obj
 0001:00002910       ?ReallocDialogItems@?$DialogBuilderBase@UFarDialogItem@@@@IAEXXZ 10003910 f i Brackets.obj
 0001:000029e0       ?UpdateSecondColumnPosition@?$DialogBuilderBase@UFarDialogItem@@@@IAEXXZ 100039e0 f i Brackets.obj
 0001:00002a40       ?SaveValues@?$DialogBuilderBase@UFarDialogItem@@@@IAEXXZ 10003a40 f i Brackets.obj
 0001:00002a90       ?MaxTextWidth@?$DialogBuilderBase@UFarDialogItem@@@@IAEHXZ 10003a90 f i Brackets.obj
 0001:00002b50       ?SaveValue@PluginEditFieldBinding@@UAEXPAUFarDialogItem@@H@Z 10003b50 f i Brackets.obj
 0001:00002b80       ?InitDialogItem@PluginDialogBuilder@@MAEXPAUFarDialogItem@@PB_W@Z 10003b80 f i Brackets.obj
 0001:00002ba0       ?TextWidth@PluginDialogBuilder@@MAEHABUFarDialogItem@@@Z 10003ba0 f i Brackets.obj
 0001:00002bc0       ?DoShowDialog@PluginDialogBuilder@@MAEHXZ 10003bc0 f i Brackets.obj
 0001:00002c20       ?SaveValue@PluginCheckBoxBinding@@UAEXPAUFarDialogItem@@H@Z 10003c20 f i Brackets.obj
 0001:00002c60       ?SaveValue@PluginRadioButtonBinding@@UAEXPAUFarDialogItem@@H@Z 10003c60 f i Brackets.obj
 0001:00002c90       ??0PluginIntEditFieldBinding@@QAE@ABUPluginStartupInfo@@PAPAXHPAHH@Z 10003c90 f i Brackets.obj
 0001:00002d30       ?SaveValue@PluginIntEditFieldBinding@@UAEXPAUFarDialogItem@@H@Z 10003d30 f i Brackets.obj
 0001:00002d60       ??0PluginUIntEditFieldBinding@@QAE@ABUPluginStartupInfo@@PAPAXHPAIH@Z 10003d60 f i Brackets.obj
 0001:00002e00       ?SaveValue@PluginUIntEditFieldBinding@@UAEXPAUFarDialogItem@@H@Z 10003e00 f i Brackets.obj
 0001:00002e30       ?CreateCheckBoxBinding@PluginDialogBuilder@@MAEPAU?$DialogItemBinding@UFarDialogItem@@@@PAHH@Z 10003e30 f i Brackets.obj
 0001:00002e80       ?CreateRadioButtonBinding@PluginDialogBuilder@@MAEPAU?$DialogItemBinding@UFarDialogItem@@@@PAH@Z 10003e80 f i Brackets.obj
 0001:00002ed0       ??_EPluginDialogBuilder@@UAEPAXI@Z 10003ed0 f i Brackets.obj
 0001:00002ed0       ??_GPluginDialogBuilder@@UAEPAXI@Z 10003ed0 f i Brackets.obj
 0001:00002f10       ?AddCheckbox@?$DialogBuilderBase@UFarDialogItem@@@@QAEPAUFarDialogItem@@HPAHH_N@Z 10003f10 f i Brackets.obj
 0001:00003040       ?AddButtons@?$DialogBuilderBase@UFarDialogItem@@@@QAEXHPBHHH@Z 10004040 f i Brackets.obj
 0001:000031a0       ?UpdateBorderSize@?$DialogBuilderBase@UFarDialogItem@@@@IAEXXZ 100041a0 f i Brackets.obj
 0001:00003250       ?AddSeparator@?$DialogBuilderBase@UFarDialogItem@@@@QAEXPB_W@Z 10004250 f i Brackets.obj
 0001:000032c0       ??0PluginDialogBuilder@@QAE@ABUPluginStartupInfo@@ABU_GUID@@1HPB_WP6GHPAXHH3@Z3_K@Z 100042c0 f i Brackets.obj
 0001:000033d0       ?AddIntEditField@PluginDialogBuilder@@UAEPAUFarDialogItem@@PAHH@Z 100043d0 f i Brackets.obj
 0001:00003490       ?AddUIntEditField@PluginDialogBuilder@@UAEPAUFarDialogItem@@PAIH@Z 10004490 f i Brackets.obj
 0001:00003550       ?AddFixEditField@PluginDialogBuilder@@QAEPAUFarDialogItem@@PA_WHHPB_W@Z 10004550 f i Brackets.obj
 0001:00003630       ?Config@@YAHXZ             10004630 f   Brackets.obj
 0001:00003ca0       _ConfigureW@4              10004ca0 f   Brackets.obj
 0001:00003cb0       ?ShowMenu@@YAHH@Z          10004cb0 f   Brackets.obj
 0001:00003dc0       _OpenW@4                   10004dc0 f   Brackets.obj
 0001:00004880       ??_U@YAPAXI@Z              10005880 f   libcpmt:newaop.obj
 0001:0000488b       ??_V@YAXPAX@Z              1000588b f   LIBCMT:delete2.obj
 0001:00004896       ??3@YAXPAX@Z               10005896 f   LIBCMT:delete.obj
 0001:000048b0       _memset                    100058b0 f   LIBCMT:memset.obj
 0001:0000492a       ??1bad_alloc@std@@UAE@XZ   1000592a f i LIBCMT:new.obj
 0001:00004935       ??_Ebad_alloc@std@@UAEPAXI@Z 10005935 f i LIBCMT:new.obj
 0001:00004935       ??_Gbad_alloc@std@@UAEPAXI@Z 10005935 f i LIBCMT:new.obj
 0001:0000495c       ??0bad_alloc@std@@QAE@ABV01@@Z 1000595c f i LIBCMT:new.obj
 0001:00004979       ??2@YAPAXI@Z               10005979 f   LIBCMT:new.obj
 0001:00004a00       __ftol2_sse                10005a00 f   LIBCMT:ftol2.obj
 0001:00004a09       __ftol2_pentium4           10005a09 f   LIBCMT:ftol2.obj
 0001:00004a1c       __ftol2_sse_excpt          10005a1c f   LIBCMT:ftol2.obj
 0001:00004a36       __ftol2                    10005a36 f   LIBCMT:ftol2.obj
 0001:00004aab       __CRT_INIT@12              10005aab f   LIBCMT:dllcrt0.obj
 0001:00004d05       __DllMainCRTStartup@12     10005d05 f   LIBCMT:dllcrt0.obj
 0001:00004d28       _free                      10005d28 f   LIBCMT:free.obj
 0001:00004d62       __VEC_memzero              10005d62 f   LIBCMT:p4_memset.obj
 0001:00004e1c       ___sse2_available_init     10005e1c f   LIBCMT:cpu_disp.obj
 0001:00004e2c       ??0exception@std@@QAE@ABQBDH@Z 10005e2c f   LIBCMT:stdexcpt.obj
 0001:00004e49       ?what@exception@std@@UBEPBDXZ 10005e49 f   LIBCMT:stdexcpt.obj
 0001:00004e56       ?_Copy_str@exception@std@@AAEXPBD@Z 10005e56 f   LIBCMT:stdexcpt.obj
 0001:00004e96       ?_Tidy@exception@std@@AAEXXZ 10005e96 f   LIBCMT:stdexcpt.obj
 0001:00004eb4       ??4exception@std@@QAEAAV01@ABV01@@Z 10005eb4 f   LIBCMT:stdexcpt.obj
 0001:00004ee9       ??1exception@std@@UAE@XZ   10005ee9 f   LIBCMT:stdexcpt.obj
 0001:00004ef4       ??_Gexception@std@@UAEPAXI@Z 10005ef4 f i LIBCMT:stdexcpt.obj
 0001:00004ef4       ??_Eexception@std@@UAEPAXI@Z 10005ef4 f i LIBCMT:stdexcpt.obj
 0001:00004f1b       ??0exception@std@@QAE@ABV01@@Z 10005f1b f   LIBCMT:stdexcpt.obj
 0001:00004f40       ??1type_info@@UAE@XZ       10005f40 f   LIBCMT:typinfo.obj
 0001:00004f50       ??_Gtype_info@@UAEPAXI@Z   10005f50 f i LIBCMT:typinfo.obj
 0001:00004f50       ??_Etype_info@@UAEPAXI@Z   10005f50 f i LIBCMT:typinfo.obj
 0001:00005028       ___onexitinit              10006028 f   LIBCMT:onexit.obj
 0001:00005059       __onexit                   10006059 f   LIBCMT:onexit.obj
 0001:00005095       _atexit                    10006095 f   LIBCMT:onexit.obj
 0001:000050ac       _malloc                    100060ac f   LIBCMT:malloc.obj
 0001:00005140       __initp_heap_handler       10006140 f   LIBCMT:handler.obj
 0001:0000514f       __callnewh                 1000614f f   LIBCMT:handler.obj
 0001:00005177       __CxxThrowException@8      10006177 f   LIBCMT:throw.obj
 0001:000051c3       __encoded_null             100061c3 f   LIBCMT:tidtable.obj
 0001:000051cc       ___crtTlsAlloc@4           100061cc f   LIBCMT:tidtable.obj
 0001:000051d5       ___set_flsgetvalue         100061d5 f   LIBCMT:tidtable.obj
 0001:00005209       __mtterm                   10006209 f   LIBCMT:tidtable.obj
 0001:00005246       __initptd                  10006246 f   LIBCMT:tidtable.obj
 0001:000052fa       __getptd_noexit            100062fa f   LIBCMT:tidtable.obj
 0001:00005373       __getptd                   10006373 f   LIBCMT:tidtable.obj
 0001:0000538d       __freefls@4                1000638d f   LIBCMT:tidtable.obj
 0001:000054bc       __freeptd                  100064bc f   LIBCMT:tidtable.obj
 0001:0000552a       __mtinit                   1000652a f   LIBCMT:tidtable.obj
 0001:000056a5       __malloc_crt               100066a5 f   LIBCMT:crtheap.obj
 0001:000056ea       __calloc_crt               100066ea f   LIBCMT:crtheap.obj
 0001:00005736       __realloc_crt              10006736 f   LIBCMT:crtheap.obj
 0001:00005784       ___crtCorExitProcess       10006784 f   LIBCMT:crt0dat.obj
 0001:000057af       ___crtExitProcess          100067af f   LIBCMT:crt0dat.obj
 0001:000057c7       __lockexit                 100067c7 f   LIBCMT:crt0dat.obj
 0001:000057d0       __unlockexit               100067d0 f   LIBCMT:crt0dat.obj
 0001:000057d9       __init_pointers            100067d9 f   LIBCMT:crt0dat.obj
 0001:0000580c       __initterm_e               1000680c f   LIBCMT:crt0dat.obj
 0001:00005830       __cinit                    10006830 f   LIBCMT:crt0dat.obj
 0001:00005a07       __exit                     10006a07 f   LIBCMT:crt0dat.obj
 0001:00005a1d       __cexit                    10006a1d f   LIBCMT:crt0dat.obj
 0001:00005a2c       __amsg_exit                10006a2c f   LIBCMT:crt0dat.obj
 0001:00005a4a       __ioinit                   10006a4a f   LIBCMT:ioinit.obj
 0001:00005c8f       __ioterm                   10006c8f f   LIBCMT:ioinit.obj
 0001:00005ce2       __setenvp                  10006ce2 f   LIBCMT:stdenvp.obj
 0001:00005f5b       __setargv                  10006f5b f   LIBCMT:stdargv.obj
 0001:00006016       ___crtGetEnvironmentStringsA 10007016 f   LIBCMT:a_env.obj
 0001:000060ad       __RTC_Initialize           100070ad f   LIBCMT:_initsect_.obj
 0001:000060d3       __RTC_Terminate            100070d3 f   LIBCMT:_initsect_.obj
 0001:000060f9       __heap_init                100070f9 f   LIBCMT:heapinit.obj
 0001:00006117       __heap_term                10007117 f   LIBCMT:heapinit.obj
 0001:00006130       __SEH_prolog4              10007130 f   LIBCMT:sehprolg4.obj
 0001:00006175       __SEH_epilog4              10007175 f   LIBCMT:sehprolg4.obj
 0001:00006190       __except_handler4          10007190 f   LIBCMT:chandler4.obj
 0001:0000631f       __XcptFilter               1000731f f   LIBCMT:winxfltr.obj
 0001:00006469       ___CppXcptFilter           10007469 f   LIBCMT:winxfltr.obj
 0001:00006489       _DllMain@12                10007489 f   LIBCMT:dllmain.obj
 0001:0000648f       ___security_init_cookie    1000748f f   LIBCMT:gs_support.obj
 0001:0000652a       __get_errno_from_oserr     1000752a f   LIBCMT:dosmap.obj
 0001:0000656c       __errno                    1000756c f   LIBCMT:dosmap.obj
 0001:0000657f       _strcpy_s                  1000757f f   LIBCMT:strcpy_s.obj
 0001:000065e0       _strlen                    100075e0 f   LIBCMT:strlen.obj
 0001:0000666b       ?_Type_info_dtor@type_info@@CAXPAV1@@Z 1000766b f   LIBCMT:typname.obj
 0001:000066e0       _strcmp                    100076e0 f   LIBCMT:strcmp.obj
 0001:00006768       __msize                    10007768 f   LIBCMT:msize.obj
 0001:0000679b       __GET_RTERRMSG             1000779b f   LIBCMT:crt0msg.obj
 0001:000067c1       __NMSG_WRITE               100077c1 f   LIBCMT:crt0msg.obj
 0001:00006970       __FF_MSGBANNER             10007970 f   LIBCMT:crt0msg.obj
 0001:000069a9       __mtinitlocks              100079a9 f   LIBCMT:mlock.obj
 0001:000069f3       __mtdeletelocks            100079f3 f   LIBCMT:mlock.obj
 0001:00006a4a       __unlock                   10007a4a f   LIBCMT:mlock.obj
 0001:00006a61       __mtinitlocknum            10007a61 f   LIBCMT:mlock.obj
 0001:00006b23       __lock                     10007b23 f   LIBCMT:mlock.obj
 0001:00006b56       ___addlocaleref            10007b56 f   LIBCMT:localref.obj
 0001:00006be5       ___removelocaleref         10007be5 f   LIBCMT:localref.obj
 0001:00006c7e       ___freetlocinfo            10007c7e f   LIBCMT:localref.obj
 0001:00006dc9       __updatetlocinfoEx_nolock  10007dc9 f   LIBCMT:localref.obj
 0001:00006e16       ___updatetlocinfo          10007e16 f   LIBCMT:localref.obj
 0001:000070b2       ___updatetmbcinfo          100080b2 f   LIBCMT:mbctype.obj
 0001:00007156       ??0_LocaleUpdate@@QAE@PAUlocaleinfo_struct@@@Z 10008156 f i LIBCMT:mbctype.obj
 0001:00007259       __setmbcp_nolock           10008259 f   LIBCMT:mbctype.obj
 0001:00007442       __setmbcp                  10008442 f   LIBCMT:mbctype.obj
 0001:000075dc       ___initmbctable            100085dc f   LIBCMT:mbctype.obj
 0001:000075fa       __calloc_impl              100085fa f   LIBCMT:calloc_impl.obj
 0001:0000767c       _realloc                   1000867c f   LIBCMT:realloc.obj
 0001:00007729       ?terminate@@YAXXZ          10008729 f   LIBCMT:hooks.obj
 0001:00007762       __initp_eh_hooks           10008762 f   LIBCMT:hooks.obj
 0001:00007773       __initp_misc_winsig        10008773 f   LIBCMT:winsig.obj
 0001:000077c8       ___get_sigabrt             100087c8 f   LIBCMT:winsig.obj
 0001:000077d5       _raise                     100087d5 f   LIBCMT:winsig.obj
 0001:00007978       __initp_misc_rand_s        10008978 f   LIBCMT:rand_s.obj
 0001:00007987       __initp_misc_purevirt      10008987 f   LIBCMT:inithelp.obj
 0001:00007996       __initp_misc_invarg        10008996 f   LIBCMT:invarg.obj
 0001:000079a5       __call_reportfault         100089a5 f   LIBCMT:invarg.obj
 0001:00007ace       __invoke_watson            10008ace f   LIBCMT:invarg.obj
 0001:00007af3       __invalid_parameter        10008af3 f   LIBCMT:invarg.obj
 0001:00007b20       __invalid_parameter_noinfo 10008b20 f   LIBCMT:invarg.obj
 0001:00007b30       __initp_misc_cfltcvt_tab   10008b30 f   LIBCMT:cmiscdat.obj
 0001:00007b60       __ValidateImageBase        10008b60 f   LIBCMT:pesect.obj
 0001:00007ba0       __FindPESection            10008ba0 f   LIBCMT:pesect.obj
 0001:00007bf0       __IsNonwritableInCurrentImage 10008bf0 f   LIBCMT:pesect.obj
 0001:00007cff       __ismbblead                10008cff f   LIBCMT:ismbbyte.obj
 0001:00007d17       @__security_check_cookie@4 10008d17 f   LIBCMT:secchk.obj
 0001:00007d30       __local_unwind4            10008d30 f   LIBCMT:exsup4.obj
 0001:00007e06       __seh_longjmp_unwind4@4    10008e06 f   LIBCMT:exsup4.obj
 0001:00007e22       @_EH4_CallFilterFunc@8     10008e22 f   LIBCMT:exsup4.obj
 0001:00007e39       @_EH4_TransferToHandler@8  10008e39 f   LIBCMT:exsup4.obj
 0001:00007e52       @_EH4_GlobalUnwind2@8      10008e52 f   LIBCMT:exsup4.obj
 0001:00007e6b       @_EH4_LocalUnwind@16       10008e6b f   LIBCMT:exsup4.obj
 0001:00007e82       ___crtMessageBoxW          10008e82 f   LIBCMT:crtmboxw.obj
 0001:00007fee       _wcscat_s                  10008fee f   LIBCMT:wcscat_s.obj
 0001:00008063       _wcsncpy_s                 10009063 f   LIBCMT:wcsncpy_s.obj
 0001:00008130       _wcslen                    10009130 f   LIBCMT:wcslen.obj
 0001:0000814b       _wcscpy_s                  1000914b f   LIBCMT:wcscpy_s.obj
 0001:000081ae       __set_error_mode           100091ae f   LIBCMT:errmode.obj
 0001:000081ed       ___free_lc_time            100091ed f   LIBCMT:inittime.obj
 0001:00008564       ___free_lconv_num          10009564 f   LIBCMT:initnum.obj
 0001:000085cd       ___free_lconv_mon          100095cd f   LIBCMT:initmon.obj
 0001:000086cb       __freea                    100096cb f i LIBCMT:a_map.obj
 0001:000088d2       ___crtLCMapStringA         100098d2 f   LIBCMT:a_map.obj
 0001:000089ff       ___crtGetStringTypeA       100099ff f   LIBCMT:a_str.obj
 0001:00008a3f       _abort                     10009a3f f   LIBCMT:abort.obj
 0001:00008a80       _memcpy                    10009a80 f   LIBCMT:memcpy.obj
 0001:00008de1       __crt_debugger_hook        10009de1 f   LIBCMT:dbghook.obj
 0001:00008de9       __fptrap                   10009de9 f   LIBCMT:crt0fp.obj
 0001:00008df2       ___report_gsfailure        10009df2 f   LIBCMT:gs_report.obj
 0001:00008f00       __global_unwind2           10009f00 f   LIBCMT:exsup.obj
 0001:00008f65       __local_unwind2            10009f65 f   LIBCMT:exsup.obj
 0001:00008fe9       __abnormal_termination     10009fe9 f   LIBCMT:exsup.obj
 0001:0000900c       __NLG_Notify1              1000a00c f   LIBCMT:exsup.obj
 0001:00009015       __NLG_Notify               1000a015 f   LIBCMT:exsup.obj
 0001:0000902c       __NLG_Dispatch             1000a02c     LIBCMT:exsup.obj
 0001:0000902c       __NLG_Dispatch2            1000a02c     LIBCMT:exsup.obj
 0001:00009034       __NLG_Call                 1000a034 f   LIBCMT:exsup.obj
 0001:00009036       __NLG_Return2              1000a036     LIBCMT:exsup.obj
 0001:00009040       __aulldvrm                 1000a040 f   LIBCMT:ulldvrm.obj
 0001:000090e0       __alloca_probe_16          1000a0e0 f   LIBCMT:alloca16.obj
 0001:000090f6       __alloca_probe_8           1000a0f6     LIBCMT:alloca16.obj
 0001:0000910c       __VEC_memcpy               1000a10c f   LIBCMT:p4_memcpy.obj
 0001:00009210       __allmul                   1000a210 f   LIBCMT:llmul.obj
 0001:00009250       _strcspn                   1000a250 f   LIBCMT:strcspn.obj
 0001:000092a0       _strpbrk                   1000a2a0 f   LIBCMT:strpbrk.obj
 0001:000092e0       ___ascii_strnicmp          1000a2e0 f   LIBCMT:_strnicm.obj
 0001:00009342       _RtlUnwind@16              1000a342 f   kernel32:KERNEL32.dll
 0001:00009360       __TI2?AVbad_alloc@std@@    1000a360     LIBCMT:new.obj
 0001:00009370       __CTA2?AVbad_alloc@std@@   1000a370     LIBCMT:new.obj
 0001:0000937c       __CT??_R0?AVbad_alloc@std@@@8??0bad_alloc@std@@QAE@ABV01@@Z12 1000a37c     LIBCMT:new.obj
 0001:00009398       __CT??_R0?AVexception@std@@@8??0exception@std@@QAE@ABV01@@Z12 1000a398     LIBCMT:new.obj
 0001:00009584       __IMPORT_DESCRIPTOR_KERNEL32 1000a584     kernel32:KERNEL32.dll
 0001:00009598       __IMPORT_DESCRIPTOR_USER32 1000a598     user32:USER32.dll
 0001:000095ac       __NULL_IMPORT_DESCRIPTOR   1000a5ac     kernel32:KERNEL32.dll
 0002:00000040       ??_R0?AVbad_alloc@std@@@8  1000b040     LIBCMT:new.obj
 0002:0000005c       ??_R0?AVexception@std@@@8  1000b05c     LIBCMT:new.obj
 0002:00000080       ??_R0?AVtype_info@@@8      1000b080     LIBCMT:typinfo.obj
 0002:00000098       ___flsindex                1000b098     LIBCMT:tidtable.obj
 0002:0000009c       ___getvalueindex           1000b09c     LIBCMT:tidtable.obj
 0002:000000a0       ___badioinfo               1000b0a0     LIBCMT:ioinit.obj
 0002:00000370       ___clocalestr              1000b370     LIBCMT:nlsdata2.obj
 0002:00000378       ___lc_time_c               1000b378     LIBCMT:nlsdata2.obj
 0002:000004e0       ___initiallocinfo          1000b4e0     LIBCMT:nlsdata2.obj
 0002:000005b8       ___ptlocinfo               1000b5b8     LIBCMT:nlsdata2.obj
 0002:000005c0       ___initialmbcinfo          1000b5c0     LIBCMT:mbctype.obj
 0002:000007e0       __mbctype                  1000b7e0     LIBCMT:mbctype.obj
 0002:000008e8       __mbcasemap                1000b8e8     LIBCMT:mbctype.obj
 0002:000009e8       ___ptmbcinfo               1000b9e8     LIBCMT:mbctype.obj
 0002:00000ae0       __cfltcvt_tab              1000bae0     LIBCMT:cmiscdat.obj
 0002:00000b08       ___security_cookie         1000bb08     LIBCMT:gs_cookie.obj
 0002:00000b0c       ___security_cookie_complement 1000bb0c     LIBCMT:gs_cookie.obj
 0002:00000b10       ___lconv_static_decimal    1000bb10     LIBCMT:lconv.obj
 0002:00000b14       ___lconv_static_W_decimal  1000bb14     LIBCMT:lconv.obj
 0002:00000b18       ___lconv_c                 1000bb18     LIBCMT:lconv.obj
 0002:00000b68       ___lconv                   1000bb68     LIBCMT:lconv.obj
 0002:00000b6c       ___globallocalestatus      1000bb6c     LIBCMT:glstatus.obj
 0002:00000b70       __pctype                   1000bb70     LIBCMT:ctype.obj
 0002:00000b74       __pwctype                  1000bb74     LIBCMT:ctype.obj
 0002:00000b78       ___abort_behavior          1000bb78     LIBCMT:abort.obj
 0002:00000b80       __NLG_Destination          1000bb80     LIBCMT:exsup.obj
 0002:00000ba0       ___mb_cur_max              1000bba0     LIBCMT:nlsdata1.obj
 0002:00000ba4       ___decimal_point           1000bba4     LIBCMT:nlsdata1.obj
 0002:00000ba8       ___decimal_point_length    1000bba8     LIBCMT:nlsdata1.obj
 0002:00000d1c       __aenvptr                  1000bd1c     LIBCMT:dllcrt0.obj
 0002:00000d20       __wenvptr                  1000bd20     LIBCMT:dllcrt0.obj
 0002:00000d24       ___error_mode              1000bd24     LIBCMT:dllcrt0.obj
 0002:00000d28       ___app_type                1000bd28     LIBCMT:dllcrt0.obj
 0002:00000d2c       ?_pnhHeap@@3P6AHI@ZA       1000bd2c     LIBCMT:handler.obj
 0002:00000d30       _gpFlsAlloc                1000bd30     LIBCMT:tidtable.obj
 0002:00000d34       _gpFlsGetValue             1000bd34     LIBCMT:tidtable.obj
 0002:00000d38       _gpFlsSetValue             1000bd38     LIBCMT:tidtable.obj
 0002:00000d3c       _gpFlsFree                 1000bd3c     LIBCMT:tidtable.obj
 0002:00000d40       __maxwait                  1000bd40     LIBCMT:crtheap.obj
 0002:00000d44       __umaskval                 1000bd44     LIBCMT:crt0dat.obj
 0002:00000d48       ___argc                    1000bd48     LIBCMT:crt0dat.obj
 0002:00000d4c       ___argv                    1000bd4c     LIBCMT:crt0dat.obj
 0002:00000d50       ___wargv                   1000bd50     LIBCMT:crt0dat.obj
 0002:00000d54       __environ                  1000bd54     LIBCMT:crt0dat.obj
 0002:00000d58       ___initenv                 1000bd58     LIBCMT:crt0dat.obj
 0002:00000d5c       __wenviron                 1000bd5c     LIBCMT:crt0dat.obj
 0002:00000d60       ___winitenv                1000bd60     LIBCMT:crt0dat.obj
 0002:00000d64       __pgmptr                   1000bd64     LIBCMT:crt0dat.obj
 0002:00000d68       __wpgmptr                  1000bd68     LIBCMT:crt0dat.obj
 0002:00000d6c       __exitflag                 1000bd6c     LIBCMT:crt0dat.obj
 0002:00000d70       __C_Termination_Done       1000bd70     LIBCMT:crt0dat.obj
 0002:00000d74       __C_Exit_Done              1000bd74     LIBCMT:crt0dat.obj
 0002:00000e80       __crtheap                  1000be80     LIBCMT:heapinit.obj
 0002:000014b8       __newmode                  1000c4b8     LIBCMT:_newmode.obj
 0002:00001614       ___mbulinfo                1000c614     LIBCMT:mbctype.obj
 0002:00001620       ___mbcodepage              1000c620     LIBCMT:mbctype.obj
 0002:00001624       ___ismbcodepage            1000c624     LIBCMT:mbctype.obj
 0002:00001628       ___mblcid                  1000c628     LIBCMT:mbctype.obj
 0002:0000162c       ?__pInconsistency@@3P6AXXZA 1000c62c     LIBCMT:hooks.obj
 0002:00001648       ___pPurecall               1000c648     LIBCMT:inithelp.obj
 0002:0000164c       ___pInvalidArgHandler      1000c64c     LIBCMT:invarg.obj
 0002:00001664       ?pArgList@UnDecorator@@0PAVReplicator@@A 1000c664     LIBCMT:undname.obj
 0002:00001668       ?pZNameList@UnDecorator@@0PAVReplicator@@A 1000c668     LIBCMT:undname.obj
 0002:0000166c       ?pTemplateArgList@UnDecorator@@0PAVReplicator@@A 1000c66c     LIBCMT:undname.obj
 0002:00001670       ?gName@UnDecorator@@0PBDB  1000c670     LIBCMT:undname.obj
 0002:00001674       ?name@UnDecorator@@0PBDB   1000c674     LIBCMT:undname.obj
 0002:00001678       ?outputString@UnDecorator@@0PADA 1000c678     LIBCMT:undname.obj
 0002:0000167c       ?maxStringLength@UnDecorator@@0HA 1000c67c     LIBCMT:undname.obj
 0002:00001680       ?disableFlags@UnDecorator@@0KA 1000c680     LIBCMT:undname.obj
 0002:00001684       ?m_pGetParameter@UnDecorator@@0P6APADJ@ZA 1000c684     LIBCMT:undname.obj
 0002:00001688       ?fExplicitTemplateParams@UnDecorator@@0_NA 1000c688     LIBCMT:undname.obj
 0002:00001689       ?fGetTemplateArgumentList@UnDecorator@@0_NA 1000c689     LIBCMT:undname.obj
 0002:000016a0       ___lconv_static_null       1000c6a0     LIBCMT:lconv.obj
 0002:000016a4       ___lconv_static_W_null     1000c6a4     LIBCMT:lconv.obj
 0002:000019cc       ___locale_changed          1000c9cc     LIBCMT:setlocal.obj
 0002:000019d0       __debugger_hook_dummy      1000c9d0     <common>
 0002:000019d4       __pDestructExceptionObject 1000c9d4     <common>
 0002:000019d8       __nhandle                  1000c9d8     <common>
 0002:000019e0       ___pioinfo                 1000c9e0     <common>
 0002:00001ae0       ___env_initialized         1000cae0     <common>
 0002:00001ae4       ___onexitend               1000cae4     <common>
 0002:00001ae8       ___onexitbegin             1000cae8     <common>
 0002:00001aec       ___mbctype_initialized     1000caec     <common>
 0002:00001af0       __FPinit                   1000caf0     <common>
 0002:00001af4       ___dyn_tls_init_callback   1000caf4     <common>
 0002:00001af8       ___sse2_available          1000caf8     <common>
 0002:00001afc       __acmdln                   1000cafc     <common>

 entry point at        0001:00004d05

 Static symbols

 0001:00004c0f       ___DllMainCRTStartup       10005c0f f   LIBCMT:dllcrt0.obj
 0001:00004f72       __onexit_nolock            10005f72 f   LIBCMT:onexit.obj
 0001:000058c7       _doexit                    100068c7 f   LIBCMT:crt0dat.obj
 0001:00005dbe       _parse_cmdline             10006dbe f   LIBCMT:stdargv.obj
 0001:00006e8f       ?CPtoLCID@@YAHH@Z          10007e8f f   LIBCMT:mbctype.obj
 0001:00006ebe       ?setSBCS@@YAXPAUthreadmbcinfostruct@@@Z 10007ebe f   LIBCMT:mbctype.obj
 0001:00006f22       ?setSBUpLow@@YAXPAUthreadmbcinfostruct@@@Z 10007f22 f   LIBCMT:mbctype.obj
 0001:000071dd       ?getSystemCP@@YAHH@Z       100081dd f   LIBCMT:mbctype.obj
 0001:00007791       _siglookup                 10008791 f   LIBCMT:winsig.obj
 0001:00007cac       ?x_ismbbtype_l@@YAHPAUlocaleinfo_struct@@IHH@Z 10008cac f   LIBCMT:ismbbyte.obj
 0001:00007dc0       __unwind_handler4          10008dc0 f   LIBCMT:exsup4.obj
 0001:000086eb       ?__crtLCMapStringA_stat@@YAHPAUlocaleinfo_struct@@KKPBDHPADHHH@Z 100096eb f   LIBCMT:a_map.obj
 0001:00008918       ?__crtGetStringTypeA_stat@@YAHPAUlocaleinfo_struct@@KPBDHPAGHHH@Z 10009918 f   LIBCMT:a_str.obj
 0001:00008f20       __unwind_handler           10009f20 f   LIBCMT:exsup.obj
 0001:00009348       ??__Fnomem@?5???2@YAPAXI@Z@YAXXZ 1000a348 f   LIBCMT:new.obj
